:020000040000FA
:100000006400F1208613D3200322E7202D307520D1
:10001000FE208620FE203A08B6003B08B70086176F
:100020008620FE203A08B8003B08B90086138620D7
:10003000FE2083164F308600831280200608F300CE
:100040008316403086008312731C3228F31C392833
:10005000731D4328F31D42288613441C5228441064
:100060001322522844140A30F107031C5228F00AC4
:1000700052284414F630F107031C3F28F00AFF30E1
:10008000F00752288617E720FE20E5200B1D4B289D
:10009000003075201928A4013A08A3003B08A200EB
:1000A00016211928E7208620FE203A0803195A282D
:1000B0000B1D5D28003075201928C201DA21D821D6
:1000C000061F6A28BF21C208031D7228213075202F
:1000D0001F211928C321C208031D7228273075204B
:1000E0005421192800307520192883169B001C14F0
:1000F0001A08831203190800922083169B0A772896
:10010000FD30F4006630F5008B28872087207E3094
:10011000F4002030F500F50F8B28F40F8B28003405
:100120000F39303EC003031D9728C10041088616D1
:10013000B500350E9C203508F200721C861172182D
:100140008615F21C0611F2180615721D861072191A
:100150008614F21D0610F219061406160000061287
:100160004230F400F40BB22800341830B300BC0164
:10017000BD01BE01BF013C3084000430B400333007
:1001800080078019F039801B0F398002840AB40B74
:10019000BF28A20DA30DA40DBF0DBE0DBD0DBC0D3E
:1001A000B30BBB28080087208612061203309C2060
:1001B000872003309C2003309C2002309C200C3090
:1001C000EF202830EF200630EF200130EA280930F8
:1001D000C0000230EC20802886129828C030EC2025
:1001E000B02806309F00831600309F003730810012
:1001F000F730850040308600831208000B11810122
:10020000BA01BB018316E73085008720F7308500EF
:1002100083120108BA00831601160000011283122E
:10022000BB0301083A0603190B290800B5208521F4
:10023000872189218B218D218F21912193294308A9
:1002400092203C080F3903192B29902089218B21FA
:1002500083218D213E293D0E0F3903193529902028
:100260008B2183218D218F213E293D080F390319D0
:100270004029902083218D218F21912111307528D3
:100280003E0E0F39031D4D29203092203E080F39B4
:10029000031D4E29203092204F298D218F2191213D
:1002A0008321932115307528430892203C080F398B
:1002B000031960299020892183218B218D216929AF
:1002C0003D0E0F3903196B29902083218B218D213D
:1002D0008F21193075283D080F3903197529902091
:1002E0008D218F218321912181293E0E0F39031DFC
:1002F0007C29203092207D298D218F2183219121FD
:1003000093211D3075282E3092283C0E90283C08F1
:1003100090283D0E90283D0890283E0E90283E08DB
:1003200090283F0E90283F089028AE239A29362324
:100330009A29E622C2043008A9003108AA0032082E
:10034000AB0008002908B0002A08B1002B08B20051
:100350002308A9002408AA002508AB0008002308E8
:10036000A9062906A906A3002408AA062A06AA06A1
:10037000A4002508AB062B06AB06A50008009721B4
:10038000F0219921CE299921E2219921F021AF2153
:100390009721F221A2219921AF219721A41FD229CF
:1003A0002D30D3292030C300A4138A22C204B528DB
:1003B000F621DB29F421F2219721A2219921EA21BA
:1003C000AF219529A221B830A5006030A400FA30F1
:1003D000A3000800A221A501A401A3010130FF2967
:1003E0007030F7293630F7293830F7293A30840051
:1003F000A221A501A4010008A300840A0008A2000C
:100400004922C204080083163E309B0083120E224C
:10041000F0000C22F100080083169B0A83161C14BE
:100420001A088312080083163E309B0070081D22B4
:1004300071081C22831208009B0A9A001C15553073
:100440009D00AA309D009C149C18242A83128C13B2
:1004500083160800AF012408031D342A2308A400D2
:100460000319442AA301AF152F08A502031D031C7D
:10047000A22B0310A41B412AA30DA40DA50B3A2AFD
:10048000A22BA61FA4130034A401A301A201A5015D
:1004900000349630A500A601A41F572AA209A3097B
:1004A000A409A20A0319A30A0319A40AA617AF01F3
:1004B0002408031D6C2A2308A4002208A300A2011B
:1004C000AF152408031D6C2A2308A400A301AF1153
:1004D0002F1624080319442A2F08A502031D031C04
:1004E000A22B0310A41B7A2AA20DA30DA40DA50B09
:1004F000722AA22B271B231C412AA21F412AA30ACE
:100500000319A40A031D412AA40CA30CA50A03196C
:100510002C2B412AA2012508031900342408A60027
:10052000A4179630A502A51FDA2AA509A50A083046
:100530002502031CB62AA500A20D2308A200240848
:10054000A300A40108302502031CB62AA500A20DB1
:100550002308A200A30108302502031CB62AA50027
:10056000A20DA2012508031D0310BF2A25080319A7
:10057000BF2A0310A40CA30CA20CA50BB92A271B9D
:10058000221CCB2A031CCB2AA20A0319A30A031993
:10059000A40AA41BDA2AA61F0034A409A309A209ED
:1005A000A20A0319A30A0319A40A0034A401A3018F
:1005B000A20100342714A71FFF34A401A61FFF3097
:1005C000A400A300A200A60DA40CFF342508031D5F
:1005D0002B080319442A24082A06A6002B08A5077D
:1005E0007E30031CF72AA50203182C2BFA2AA50239
:1005F000031CA22B2408A2002308A100A217AA17FB
:100600000310A401A3011030AF00211C0D2B2908F9
:10061000A3072A0803182A0FA407A40CA30CA20CF2
:10062000A10C0310AF0B052BA41B1A2BA20DA30DBD
:10063000A40DA503271B231C292BA21F292BA30ACA
:100640000319A40A031D292BA40CA30CA50A031942
:100650002C2BA61FA4130034A714A71FFF34FF30B0
:10066000A500A400A300A60DA40CFF342B080319B9
:10067000AC2B25080319442A24082A06A600A4172F
:10068000AA17AF012408A2002308A1002908A1028B
:100690002A08031C2A0FA202A201A101031C562B47
:1006A0000310A40CA30CA20C0130AF002B08A50270
:1006B000031C602B7E302F07A50703182C2B652BFE
:1006C0007E302F07A507031CA22B1030AE00A10D12
:1006D000A20DA30DA40DAF0D2908A3022A08031C27
:1006E0002A0FA4022A0DAF042F1C782B21147F2B74
:1006F0002908A3072A0803182A0AA4072110AE0B09
:10070000672B271B211C9B2B0310A30DA40DAF0DE2
:100710002908A3022A08031C2A0FA4022A0D2F0469
:100720000139A1070318A20A031D9B2BA20CA10CDF
:10073000A50A03192C2BA61FA2132208A400210826
:10074000A30000342715A71FFF340130A500A40122
:10075000A301A60DA40CFF34A715FF348030AA0610
:1007600024082A06AF00A201A80125082B02031CB9
:10077000CB2B2B08A0002508AB002008A5002A08D9
:10078000A0002408AA002008A4002908A00023082B
:10079000A9002008A3002B08031900342408A60090
:1007A000A417AA172B082502AB000319F12B083058
:1007B0002B02031CE82BAB002908A8002A08A9007B
:1007C000AA0108302B02031CE82B2608A4000034E1
:1007D0002B080319F12B0310AA0CA90CA80CAB0BC6
:1007E000EB2BAF1FFB2BA809A909AA09A80A03191B
:1007F000A90A0319AA0A2808A20729080318290F19
:10080000A3072A0803182A0FA407AF1B0F2C031CE9
:100810007A2AA40CA30CA20CA50F7A2A2C2B03185D
:10082000572AA209A309A409A20A0319A30A0319B2
:08083000A40A8030A6062A2A62
:02400E00623F0F
:104200002000200020004F00760065007200200092
:10421000520061006E006700650020002000200051
:10422000000020006E0046000000200070004600E4
:10423000000020006D0048000000200075004800CC
:1042400000002000430020003D002000000020006E
:104250004C0020003D002000000020002000200035
:10426000430061006C00690062007200610074002C
:1042700069006E0067002000200000002700100089
:00000001FF
